:100000002CC054C053C052C051C051C04FC04EC08C
:100010004DC04CC04BC04AC049C048C047C000009A
:1000200000000000000000000000000023456C9864
:10003000C9FF040714233764A0FFFFFFFFFFFFFF82
:10004000FFFFFFFFFF000000000000000000234052
:100050005F7AB4FFFFFFFFFFFF0011241FBECFE553
:10006000D2E0DEBFCDBF20E0A0E6B0E001C01D922F
:10007000A638B207E1F7E1E6F0E085E5808781E0A8
:1000800083831482128286831182ACE6B0E08EEF05
:1000900015968C9315978DEF17968C938BE081872F
:1000A00088E58287612C712C7ED0BCC0A9CF1895C1
:1000B00025B7277E25BF29B7226029BF21E022BFAF
:1000C000019728F020E188952150E9F7F9CF0895AC
:1000D00088EE93E0EDCF81EA87B986EC86B9369A4F
:1000E0000895369A3699FECF85B10895811104C0DE
:1000F0001BBC19BC18BC0895815090E0FC01E25E65
:10010000FF4FE491EBBDFC01EE5CFF4FE491E9BDD4
:10011000FC01EA5BFF4F849188BD08950F931F9304
:10012000CF93C82F8B01CC2369F085E0DFDFC801B6
:10013000BFDF1BBC19BC18BCC801BADFC801B8DFDF
:10014000C150F1CFCF911F910F910895CF93DF93BD
:10015000D82F64E170E08AE0E1DF84EF91E0A8DF6E
:100160008D2F64E653D0CAE06C2F50D0892F68ECF5
:1001700070E0D4DFADDF8D2F6C2F48D0D92F46D063
:10018000892F68EC70E0CADFA3DF68EC70E08D2F88
:10019000C5DF9EDF64E170E08AE0C0DF84EF91E0BC
:1001A000DF91CF9185CF83EA87B986EC86B93699FE
:1001B000FECF369A3699FECF85B18FE384BBBB9ACA
:1001C000C39AB99AB89ABC9A81E08ABD83BF9AB59E
:1001D00090629ABD9AB590689ABD9FEF9DBD80BF11
:1001E00080E68CBD97B328B3892F90E080959095D9
:1001F0008B7F822B88BB85B7806285BF78946BDF4D
:100200008CE291E055DF6DDFA1DFFACF991B79E039
:1002100004C0991F961708F0961B881F7A95C9F796
:0802200080950895F894FFCFCA
:00000001FF
